:020000020000FC
:040000000C948200DA
:1001000000EC05BFC0EDD0E000E003500DBF01E002
:1001100000400EBF0E945101002309F424D0E0E604
:10012000F0E002E010E00E94D616E0E0F0E000E02F
:1001300010E040E050E00E94C816E4E0F1E00CE579
:1001400013E00E94D616E2E5F2E000E011E044E0A0
:1001500050E00E94C816EAE6F1E000E614E040E054
:0A01600050E00E94C8160C945301F1
:0402A20001E00895DA
:1002A6000E946E07002319F40E948503FDCFF8947F
:0C02B6000E94B60178940E94D501FDCF93
:10016A000A53494F32494445207665722E20332E70
:10017A00322028632932303032204D4D536F667455
:10018A0020666F722041544D454C2041546D65677D
:06019A00613136310A005C
:1002C20009B1073119F408E009B9089507E109B93C
:1002D200089557980093060210930702002700938F
:1002E200040200930502E0E6FF27F083579A08957F
:1002F20012D0015010400C5F1E4FE02FF12F80836F
:10030200E0E6FF2720E630E0082F11274081040FA6
:100312001F1F11500895E4E0F2E0008111810F5F88
:100322001F4F00831183089519B71D7F19BF0093D2
:100332000A0209B7026009BF089509B70D7F09BF14
:1003420000910A02002311F0002701C001E019B751
:10035200126019BF08950EEFE7DF04E010E0B9DF85
:10036200949A01E00093080208958C9A909A07E10A
:1003720009B908E90AB98A98929A07EB02BF05E01F
:1003820003BF09B7026009BFE6CF000F111F202F7C
:10039200312F01501040232B11F00000F8CF0895A7
:1003A2005D9BFECF0CB908950E94EA16A4E0B1E06D
:1003B200C4DF002311F084DFCEDF00910802E6E5FE
:1003C200F2E00C946B16829B9CC00EEFADDFEA2F1D
:1003D200FB2F41810A2F1B2F0E949007002309F453
:1003E2008FC00027009309029AD0E056FE4FC895AD
:1003F200002009F483C093D0E056FE4FC895EA2F3F
:10040200FB2F01810016E1F48AD094D00029C1F0BB
:1004120086D090D0E02FF02D46E052E00A2F1B2F1D
:100422000995002369F07BD0ED55FE4FC8950092E7
:10043200080200910602109107024BDF949861C0F6
:10044200009109020395CECF08EC10E05DD009F4CB
:100452004CC065D0EC55FE4FC89562D009F445C03A
:1004620003E49EDF07E034C040C03FC00AEF10E063
:100472008CDF7DD018F567D0EC5FFE4F008190DFF6
:1004820000E610E060D0EC5FFE4F20813327E0E60B
:10049200FF274081240F311F315055D028F0EC5FE7
:1004A200FE4F2081239503C0EC5FFE4F2081E02F99
:1004B200F12F0081020F00832EDFDBCFE0E6FF2762
:1004C20000811DC03ED002E02FDF01E469DF04E0BD
:1004D2000093080216C000ED17E016D031F01FD0CD
:1004E200EC55FE4FC8951CD021F405E408C029D074
:1004F20039D003E404C004EF11E047DF0EE450DF1B
:100502002ADFE4E00C94FB1640DF2CD021D0EC551E
:10051200FE4FC895002D3196C8950029089518C040
:10052200002D3196C895E02FF02D04E011E00995D9
:1005320000230895EF55FE4FC895002D3196C895BA
:10054200089508EC12C0E0910402F09105020895AA
:1005520000910902112746E050E00E94CC15E02FDD
:10056200F12F089501E41CDF0AEF10E00ECF009195
:10057200040210910502209106023091070202172F
:10058200130708950A921A922A923A920A931A9398
:100592002A933A934A935A936A937A93EA93FA93F1
:1005A200FFB7FA938A938CB182991AC0009108021C
:1005B2000130B1F445D050F49BDE082F08F00395CA
:1005C200E22FF32F1081100F10830AC0E0E6FF27FD
:1005D2000081081711F402E001C008E0009308024C
:1005E200829B1CC0009108020430C1F429D048F457
:1005F2007FDE08F08395E22FF32F0081080F00833E
:100602000DC00EEF91DEE0E6FF270081081711F41E
:1006120005E002C055DE09E0009308028991F991D4
:10062200FFBFF991E9917991699159914991399174
:100632002991199109913990299019900990189549
:1006420002E072DE94CF0A93EA93FA93FFB7FA9329
:1006520000910A020E3F49F000910A02002329F09C
:1006620000910A02015000930A0207EB02BFF991BE
:0A067200FFBFF991E9910991189575
:10025600020082020900E401630282026C022502A6
:08026600370281027C027802DC
:04002C000C94240309
:040034000C94C30263
:10067C00000F111F221F331F35D001501040204096
:10068C003040452B462B472B11F00000F5CF089539
:10069C002ED00E942E16742E7394082F192F2A2FE9
:1006AC003B2FE42D24D00E942E16E42D23D00E9443
:1006BC002E16642E2A2F3B2FE42D038114814281A8
:1006CC0055270E94CC15402F512F66277727082FCE
:1006DC00192F0E942E16402E512E062D0F700056EB
:1006EC00602E0895402F512F622F732F0895438150
:1006FC00548102C04281552766277727089500EA66
:10070C0016E821E030E0B4DFAD9800E41DE023E012
:10071C0030E0AEDFAD9A089531E040E81127332385
:10072C0039F0202F232309F0142B330F4695F7CFE4
:10073C00012F08959A938A93902F042F852FECDF25
:10074C001FEF1ABB17BBF89415B3107E192B15BBF2
:10075C00AF980BBB88BBAF9A000005B30F6105BB0C
:10076C0078940FEF0ABB0BBB07BB08BB899199911F
:10077C0008959A938A9311271ABB1FEF1BBB11275D
:10078C0017BB1FEF18BBF89415B3107E102B15BBBD
:10079C00AE980000AE9A09B386B315B31F6115BBB2
:1007AC0078941FEF1ABB1BBB17BB18BBB5DF182FF8
:1007BC008991999108950E94EB16A02F80E197E200
:1007CC00AA2339F00197082F092B19F4AD980027AB
:1007DC0005C00DE1CEDF00309CF301E0E3E00C94AA
:1007EC00FC160E94EA16802FA0E1B7E2882339F0AC
:1007FC0011970A2F0B2B19F4AD98002705C00DE1AA
:10080C00B8DF03FFF3CF01E0E4E00C94FB160DE13D
:10081C00B0DF00FF03C0AD9801E00895AD9A00274A
:10082C00089525D0B0F0E42DF52D01850030042F6E
:10083C002CF0152F262F372F2BDF01C028D011D0ED
:10084C0041F02ED041E209D021F03ED011F401E06C
:10085C0001C00027E8E00C94F71650E00DE16ADFC8
:10086C0036C005E086DF01E0A6DF002308950E9474
:10087C00E616402E512E842F952FA62FB72FE02F42
:10088C00F12F29D004171507260737070895702E66
:10089C00492E5A2E6B2E0FE0602200EE600E08954A
:1008AC00462D552709E146DF41E050E009E042DFE3
:1008BC00472D55270DE03EDF442D552701E13ADF4A
:1008CC00452D50E005E136CFA2DF0023089501E06D
:1008DC0088DF0023089505811681278130850895CE
:1008EC00C6DFB8F0E42DF52D018506FD12C0E42D10
:1008FC00F52D01850030082F2CF0192F2A2F3B2FB6
:10090C00C7DE01C0C4DFADDF21F0CADF41E3A5DFE4
:10091C0011F4002701C001E0E8E00C94F716082F51
:10092C00192F2A2F3B2F42E00C9425160E94EA1611
:10093C00802F912F2AD0A0E0B1E0E02FF12F21855C
:10094C0026FF0EC0222733273A932A937A936A9371
:10095C005A934A93402F512F082F192F54D112C05C
:10096C0060DF002371F00A2F1B2F1197012B01E080
:10097C0049F0FFDEE82FF92F019311938E2F9F2F53
:10098C00F2CF0027E8E00C94FB16042F152F4C81B6
:10099C005D816E817F8108950E94EA16A02FB12F90
:1009AC00F4DF80E091E0E02FF12F218526FD12C0CD
:1009BC0097DF002379F0082F192F0197012B21F0D5
:1009CC004D915D910ED0F7CF0ED021F07DDF11F45B
:1009DC0001E001C00027E8E00C94FB16A02FB12F1A
:1009EC0040CF01E0A7CE01E03FCF0E94E816F6DF32
:1009FC0009F46AC071D04CEE30DF09F465C064DFD5
:100A0C0009F062C04424552401E0501608F042C09D
:100A1C005FD0042D152DEEE6F2E00C946F1600E07D
:100A2C009030A4F552C0EA2FFB2F808391832EC007
:100A3C00EA2FFB2F82832AC0EA2FFB2F8383948318
:100A4C0025C091FF23C0EA2FFB2F01850068018789
:100A5C001DC0EA2FFB2F01850030C4F422278583AB
:100A6C0096832783208712C0EA2FFB2F0185003045
:100A7C006CF411274581568167817085410F511F98
:100A8C00681F791F45835683678370870FEF401A61
:100A9C00500ABACFEA2FFB2F018500309CF0008161
:100AAC0011812227332726DE0E940016EA2F1FDE33
:100ABC000E940016EA2F14D00EDF01501040204087
:100ACC0030400ED001E001C00027E6E00C94F9168E
:100ADC0050DE802F912F089540EA50E009E12ACE94
:100AEC0005831683278330870895BBDE11F4002716
:100AFC000895F2DF4CE050E001E11BD005E119D084
:100B0C0005E017D009E015D00DE013D001E112DE9D
:100B1C0048E050E005E10EDE40EA9FDE11F40027CC
:100B2C00089561DF11F40027089501E0089550E065
:100B3C0001E000DE4427552708950E94E016A02E00
:100B4C00B12E442E552E662E772E88889988AE8528
:100B5C00BF85CC2404E0D02EC8DF002309F449C0A3
:100B6C0048EA50E03EDF472D562D3BDF452D542DF6
:100B7C00DFDF37DF40E051E034DF3FD0D1F1002739
:100B8C0030DE0023B1F1A0DEA1F52C2D3D2D0FEFB1
:100B9C00C00ED01E232B01E011F19ADF0A2F0B2B74
:100BAC0011F011970BC0082D092941F00FEF800EA1
:100BBC00901EEA2DFB2D8193AE2EBF2E0A2F0B2BF0
:100BCC0011F01197E2CF082D0929F9F20FEF800EE1
:100BDC00901EEA2DFB2D9193AE2EBF2ED6CF01DEAB
:100BEC00002329F001E0C5DD72DEE1F702C001E06F
:100BFC0001C00027E2E10C94F1164427552701E0CF
:100C0C0099DD002731CE0E94E616602E712E4C84A1
:100C1C005D8488859985AA85BB85E42FF52F018590
:100C2C0006FF58C058DE80179107A207B30708F0DB
:100C3C0051C001E0401602E0500608F04BC0042DF4
:100C4C000529B9F1082F0370112722273327033008
:100C5C0010402040304069F562DE802F912FA22F8A
:100C6C00B32F00E012E0041915091A930A93042D0E
:100C7C00152D1A5F1A930A93482F592F622F732F31
:100C8C002FD009F427C08F5F9F4FAF4FBF4F5A92A1
:100C9C004A92002711271A930A93482F592F6A2F2B
:100CAC007B2F64187508600E02E0701E19D0A1F439
:100CBC0011C000E012E01A930A93082F0370102F52
:100CCC000027110F040D151D1A930A9328DE0ADD57
:100CDC0007D011F4002701C001E0EEE00C94F716E8
:100CEC00062D172D2ADF002308959A938A931A93C1
:100CFC000A93842FFADE002369F04BE151E018DFF0
:100D0C0070DE482F50E014DF13DF6BDE76DF11F05E
:100D1C00DBDD11F0002701C001E022968991999149
:100D2C00089542E0E2CF43E0E0CF0E94EA1656DE9F
:100D3C0069F1D2DE41EA91DD49F1C6DD39F588274A
:100D4C00992701E09130B0F414DD282F392F205071
:100D5C00304021F02153304021F00AC0103044F0D3
:100D6C0015C011FF13C0EA2FFB2F01850068018706
:100D7C000196E7CFEA2FFB2F01850064018700E87D
:100D8C0011E327E130E0ACDE01E001C00027E4E034
:100D9C000C94FB160E94E616402E512E642E752ED6
:100DAC00A4DE002319F143E0C2DE1BDE42E1BFDE0C
:100DBC00BFDEBEDE16DE17DEC9F089DDB9F084DDDC
:100DCC00A9F4AA27BB27EA2FFB2F399701E078F467
:100DDC007FDE0A2F1B2F0650104031F4E42DF52D29
:100DEC008083E62DF72D90831196EDCF0027E8E058
:100DFC000C94F7162297E02FF12F018506FF12C0F5
:100E0C004C2F5D2F4F5F5F4F0C2F1D2FC3DF002327
:100E1C0049F00881E8E8F2E00C946B1601E003C09D
:100E2C00002701C002E0229608959A938A93802F9E
:100E3C00912F0027E82FF12F008301830283038376
:100E4C00048305830683078300870187082F6DDFE2
:100E5C000023082F192F41F066DF082F192FCADF46
:100E6C000130D9F702E006C0C0DD002311F001E02B
:100E7C0001C000278991999108952EDE4EE050E033
:100E8C000AE158DC0AE010E020E030E0F1DB4AE057
:100E9C0050E00AE14FDC00E211EA27E030E0E8DB49
:100EAC00002789CC9A938A93802F912F0FEF0ABB3E
:100EBC000BBB07BB08BB04BB0FE105BBAE9AAF9ADB
:100ECC00AD98DBDF082F192FB0DF89919991089528
:10026E000000014C051505011905021E05032205A6
:10027E002B27050B2F05013A05FB00011807140764
:10028E00021807021807241807011807111607C5C8
:03029E001807FB43
:100EDC008D988E988F98959A969A979A00B3003021
:100EEC008B9A14F0939801C0939AE1E6FF27F08354
:100EFC000E946F14002321F48B9A939A0027089573
:100F0C0000B300300CF08B9A939A01E0E1E6FF27D6
:100F1C0000830895E02FF12F2081213711F4859B58
:100F2C0007C0E02FF12F2081223701F5859B1EC0D1
:100F3C004131C1F04231B1F04631A1F0433191F071
:100F4C00443181F0453171F0473161F0483151F055
:100F5C00493141F04A3131F04B3121F04C3111F033
:100F6C004D3111F401E0089500270895E02FF12F81
:100F7C002081213318F02081293310F000270895A7
:100F8C0020B320303CF4E02FF12F2081213311F4D9
:100F9C000027089586990EC0E02FF12F2081213370
:100FAC0011F422E306C0E02FF12F2081223311F43B
:100FBC0021E32083E02FF12F008100530E943E1289
:100FCC00012B11F001E0089500270895E02FF12F77
:100FDC002081205320930B022381028100930C0269
:100FEC0020930D0200910B020E943E1220910C02E4
:100FFC0030910D0202171307089508D00CE00DD0A4
:10100C0000910B020E943E12012B0895E02FF12F4C
:10101C000081005300930B02089510E0E42FF52F8C
:10102C000083118308951DD031F0D0DF20F0022F02
:10103C00132F032B11F4002711C0E22FF12F31973E
:10104C0038F0E22FF12F349718F400E810E001C0CB
:10105C0015D0E82FF92F0083118301E08991999124
:10106C0008959A938A93842F952FE1E6FF27208188
:10107C00222308959A938A93802F912F00910B022B
:10108C000C942C1202D00C944E131A930A93409188
:10109C000C0250910D0200910B020895E2DF31F029
:1010AC0095DF20F0022F132F032B11F4002711C012
:1010BC00E22FF12F319738F0E22FF12F349718F4FB
:1010CC0000E810E001C0DADFE82FF92F008311836C
:1010DC0001E0899199910895D8DF0C94D31296DF91
:1010EC0004E00FD00AD0012B11F400270895E1E69B
:1010FC00FF27008108958E2F9F2F00910B020C94D7
:10110C003E128BCFB7DF0030114011F400E301C069
:10111C0000E1E82FF92F01930FEF019300EE0193FB
:10112C000027008301E089919991089566DFF9F613
:10113C0000270895DCCF9A938A93802F01E0E82F43
:10114C00F12F019300E10193D6DFE82FF92F1193D2
:10115C00D2DFE82FF92F0193002701938E2F9F2FB9
:10116C008DDF0030114041F40CE0E82FF92F019392
:10117C0001E00193002707C008E0E82FF92F019345
:10118C000027019300E8019300E4019309E4019323
:10119C0004E4019305E4C5CF30DF09F0A8CF0027A4
:1011AC000895A5CF9A938A93E02FF12F8281982FDF
:1011BC000381802FA2DF0817190711F0002701C047
:1011CC0001E08991999108959A938A93842F952F90
:1011DC001DDF0E942C12E82FF92F00831183008150
:1011EC001181012B11F4002703C0E1E6FF270081D8
:1011FC008991999108953EDF025010402FEFE82F0E
:10120C00F92F21932193202F312F01501040232BA4
:10121C0009F488CF2227F6CF85CF1A930A9301E0E1
:10122C0070DFE1E6FF270081229608952AE0E02F87
:10123C00F12F208301E00895E02FF12F028100931C
:10124C000B020FE05EDF00910B020C942412402F76
:10125C00512F00910B020C944811EECF402F512FBF
:10126C0000910B020C9473111A930A930FE0D8CFD0
:10127C000C941811F9CF0C94341121E030E0E42FC8
:10128C00F52F20833183E02FF12F02810C9406126D
:10129C002FEFE02FF12F20832ACF1A930A9301E02E
:1012AC00BFCF2FEFE02FF12F20830C9452121A9303
:1012BC000A930AE0B5CF0E94BB1201E008951A937D
:1012CC000A9304E0ADCF0E94C11201E00895CCCF87
:1012DC000C94C010C9CF0C94D310C6CF0C94E3104F
:1012EC00C3CF0E94F01001E00895BECF9A938A9369
:1012FC00802F912F0E94D613002339F0082F192F1D
:10130C000E94F0100E9414110DCF0FE010E01A9300
:10131C000A9344275527082F192F0E94411702CFF3
:1001A00053750806880850190803480857190803AA
:1001B00048085254080672084E9C0806A1084FD2FF
:1001C0000803D80821EA080601093F1309061C099B
:1001D000112209062D09123309033409133A0906BD
:1001E0003E091440090641091653090657091543EB
:1001F00009064E09175D09066109186509066909AE
:10020000196D09066E091A70090671091B73090335
:1002100074091C76090677091D7B09067C09000014
:0402200000010000D9
:10132C000E94EA16802F912FA22FB32FE0E0F1E05C
:10133C0061D069D089F0BA93AA939A938A936CD0AE
:10134C000E949C04002311F4002707C0E0E0F1E0A8
:10135C0080839183A283B38301E0E4E00C94FB16B9
:10136C000E94EA16802F912FA42FB52F5AC0222746
:10137C00332701505CD05FD0802F912FA22FB32F39
:10138C00082D5FD0E25FFB4F0081118122813381F8
:10139C00800F911FA21FB31F0895041B150B260B62
:1013AC00370B40914A045527662777270E942E1643
:1013BC00802F912FA22FB32F8E5F9F4FAF4FBF4F18
:1013CC000895802F912FA22FB32F823000E01007A9
:1013DC00200730070895802F912FA22FB32F0F3F96
:1013EC001F4F08950E94E616602E712E442E552E26
:1013FC00E5E5F4E0008111812281338108958F5F4E
:10140C009F4FAF4FBF4F80179107A207B3070895A7
:10141C003A932A931A930A934BE454E00EE012E0A9
:10142C0008954CEC5DE09CD20023089502501040CE
:10143C00204030400895442D552D662777270C9475
:10144C002E16112747E050E00E94CC15E02FF12F0B
:10145C0008955A934A93DCDF0C940906D9DF0C9457
:10146C00D2040E94EA16802F012F122F232F33272C
:10147C0031D019F40027112705C0E82FFF2734D0ED
:10148C000081118122273327E4E00C94FB16082FEE
:10149C00CDDF40914A045527662777270E94001616
:1014AC0035D03BC0E8E3F4E03DC0E8E3F4E005846C
:1014BC0016842784308881859285A385B485081687
:1014CC0019062A063B06089521D0401751076207DA
:1014DC0073070895E8E3F4E04181528163817481DC
:1014EC001CD01EDF00230895EE0FFF1FE25FFD4F9F
:1014FC000895E8E3F4E00584168427843088E5E554
:10150C00F4E000821182228233820895E8E3F4E051
:10151C0045815681678170850895040F151F261F1C
:10152C00371F0895018512852385348508950E94FF
:10153C00EA16802F47E00E942516CCDF29F40027FD
:10154C0011272227332708C0E82FEF77FF27EE0F4C
:10155C00FF1FCADF4FDF3F70E4E00C94FB160E94C4
:10156C00E616602E712EE02FF12F44DFADDF28F44C
:10157C00E62DF72D3FDF11DF01C050D04424552458
:10158C0000913804045039F0025029F00650E9F06B
:10159C000357B9F139C0082F192F2A2F3B2F61DFC0
:1015AC00402F412B422B432B79F14FEF441A540A15
:1015BC000F3F140740E02407340711F020DF21F51A
:1015CC000ADF2040304039F719C0082F192F2A2F75
:1015DC003B2FADDF402F412B422B432BA9F04FEF7C
:1015EC00441A540A0F3F140724074FE0340711F034
:1015FC0006DF51F4F0DE2F4F3F4039F7042D152D47
:10160C000AC001E010E007C0E62DF72D068100624C
:10161C00068300271127E8E00C94F71682E090E08F
:10162C00A0E0B0E0089511D0065F1F4F0E946F1527
:10163C000051FDDE442D552D662777270C942E1670
:10164C00042D152D262D372D089500915B04109136
:10165C005C0408950E94EA16802F912FA42FB52FB9
:10166C00C7DE56DF3CD090F500915904112745E0B8
:10167C000E94DC15025F1D4F00935E0410935F0403
:10168C00009159040031E0F4B5DE32D011F400279A
:10169C001EC000915904039500935904082F192F6B
:1016AC00EA2FFB2F0995002311F001E010C0E5E5AE
:1016BC00F4E001851285005E1F4F01871287E0CF91
:1016CC0000270093590496DE05D0CACF02E0E4E06F
:1016DC000C94FB160F5F1F4F2F4F3F4F11C0041779
:1016EC001507260737070895082F192F2A2F3B2F88
:1016FC00F8CE018712872387348707C0E5E5F4E02D
:10170C0000831183228333830895058716872787E7
:10171C00308B08959FDF002339F00A9519F00A9554
:10172C0019F002C001E00895002708950E94EA16FE
:10173C00A02FB12F842F952FB5DEE0DF0DD01BD05D
:10174C0018D0002700935904482F592F0A2F1B2F0C
:10175C00E1DFE4E00C94FB1600914A041127409160
:10176C00490455270E94CC15212F210F220B322F13
:10177C000895D3DE05C04081518162817381089543
:10178C00058316832783308708952CDE9DDE10F4A5
:10179C0004DE01C043DF3FD039F00A9519F00A95F9
:1017AC0029F004C001E011C000270FC0082F192F29
:1017BC002A2F3B2F56DE05DE10F069DE01C072DEEB
:1017CC0007D000E0A007B00731F7E8E00C94F7165B
:1017DC0095DF00914A04112722273327CCDF9DDEA9
:1017EC00CFDF8F3F0FEF90070895442D552D0E94AA
:1017FC00EA1541505040042F152F462D572D0C94AF
:10180C00CC15442D552D0E94EA15452B082F192F68
:10181C002A2F3B2F0895442D552D062D172D1ADFF9
:10182C000023089504D0B1DFE4E00C94FB160E9471
:10183C00EA165FDE00904A041124222433248081AE
:10184C009181A281B381080E191E2A1E3B1E0582AE
:10185C001682278230862227209359040895C2DDF0
:10186C0033DE10F49ADD01C0D9DED5DFB9F00A956C
:10187C0019F00A9521F003C001E011C00FC0082F28
:10188C00192F2A2F3B2F53DE9CDD10F000DE01C0F8
:10189C0009DE9EDFA0070FE0B00739F70027E8E06C
:1018AC000C94F716C4DFDBDFE4E00C94FB160E940B
:1018BC00E816802F912F442E552E9ADD19DFF1F06A
:1018CC000091590410915A04025F1D4F39D0B1F0A8
:1018DC003FD00E94441511272091590430915A048D
:1018EC00020F131F125098F0422F532F81DDB1DDE0
:1018FC00002321F00EE012E023D011F4002710C0D9
:10190C0012D0132F1170158375DDE4DE01C00BD0DE
:10191C00082F192FE42DF52D0995002371F201E004
:10192C00E6E00C94F91691DE0E9444151127E5E5CA
:10193C00F4E024813581200F311F248335830895F1
:10194C0000935B0410935C040E94441500230895DB
:10195C007CCECFDD22272093590420935A04A7CFA5
:10196C000E94EA1620913804245039F0225029F0B4
:10197C00265049F0235749F00AC097DD11F4D6DE02
:10198C0007C050DF05C08EDF03C0E3DF01C00027B6
:10199C00E4E00C94FB160E94EA16209138042450C3
:1019AC0039F0225029F0265049F0235749F00AC04B
:1019BC007CDD11F4AFDE07C0E8DE05C050DF03C0EC
:1019CC0076DF01C00027E4E00C94FB160E94E216BF
:1019DC00802F912F842E952EAC84BD84E02FF12F77
:1019EC00B0A170D040E250E0082D192D0E94411793
:1019FC0003E069D040E250E00A2D1B2D0E944117F4
:101A0C00BB2309F445C0BF3008F042C0E82FF92FC2
:101A1C0001A10230E8F1482E592E01E2400E00E0FF
:101A2C00501E6B2EAA274BE337D031F057D020F441
:101A3C00B02F082F0F5DB01BBD3050F54EE22CD0EF
:101A4C0069F04CD058F4602E282F2F5D621A0F5F6E
:101A5C001F4F402E512EAB2FA619AA9509E06016E8
:101A6C00B8F4A430A8F477247A926A928196482F1D
:101A7C00592F082D192D0E942A17BB27BA93AA9308
:101A8C00442D552D0A2D1B2D0E942A1701E001C053
:101A9C000027EEE00C94F31650E0082F192F0F5D81
:101AAC001F4F0E945217202F212B0895402F512F8A
:101ABC00622F732F062D172D24D0402E512E012B63
:101ACC0008951AD008E010E01A930A9308950E9422
:101ADC002A17082D192D2A2D3B2D0895282F392F23
:101AEC002F5D3F4F402F512F421B530B4B17504034
:101AFC0008950F5F1F4F28CF0087118722873387E8
:101B0C0008953FD0042F152F262F372FF1DD49F1E3
:101B1C002EE032E000910E0210910F0206391240B5
:101B2C0029F0E82FF92F068500610687E22FF32FA5
:101B3C00048115810030114029F4E82FF92F068516
:101B4C0000640BC0E22FF32F048115810038104084
:101B5C0029F0E82FF92F06850061068749DCC8DDDE
:101B6C0019F4002711270AC0E82FF92F068506FF64
:101B7C0003C000E011E002C000E810E089919991E7
:101B8C0008959A938A93802F912F08950E94E216BC
:101B9C002397602E712E0FE096DF44275527062DD4
:101BAC00172D0E944117009138040F3709F062C0BD
:101BBC00CFDEF6D0012B022B032B09F4ACC0C8DE10
:101BCC0098DF09F0A8C00C2F1D2F1A930A93462DED
:101BDC00572DBEDEFBDE002309F49DC0E0915B04B3
:101BEC00F0915C04018D01FD96C0E62DF72D068564
:101BFC000460068703E067DF41E352E00C2F1D2FE2
:101C0C000E5FDED069F4A4DECBD001301240204050
:101C1C00304008F080C008E0E62DF72DBCD024C081
:101C2C0003E051DF44E252E00C2F1D2F0E5FC8D0B1
:101C3C0009F071C08DDE0E5F1F4F0E946F1536DFED
:101C4C0009F469C0F0DC452B462B472B41F080DEB4
:101C5C00A7D0013011402040304008F05CC0E3DCDC
:101C6C00E62DF72D0487158773DE9ED0E62DF72D14
:101C7C0043DF8CC0AAD0828C938C04891589A02E4A
:101C8C00B12E0081053E09F446C00081002309F401
:101C9C0042C003850E7DF9F5048D158D268D378D8B
:101CAC00012B022B032B09F436C003E00CDF41E3BC
:101CBC0052E081D0C9F489D0048D158D268D378DD5
:101CCC00013012402040304030F508E0E62DF72D71
:101CDC000687002711270487058702E080169106E6
:101CEC00A106B106F0F546C003E0EDDE44E252E099
:101CFC0062D089F46AD0038500FF05C0E62DF72D6C
:101D0C0006850460068766D018F0E3DEC1DB01C0EF
:101D1C00C9DBCCDE11F400273AC057D0848D958DE9
:101D2C00A68DB78D082F192F2A2F3B2F81DC452B21
:101D3C00462B472B39F0813001E0900700E0A007DB
:101D4C00B00728F580519040A040B040082F192FC3
:101D5C002A2F3B2F70DBE62DF72D048715873AD001
:101D6C0048F00EEF800E0FEF901EA01EB01EB1DEDD
:101D7C0090DB01C097DBE62DF72DA3DE40915E04CE
:101D8C0050915F04062D172D0E942A1701E023960F
:101D9C00ECE00C94F316068700270487058708955A
:101DAC00065F1F4F0C946F150E5F1F4F0E946F152F
:101DBC0042E00C941C1600915E0410915F04085FC5
:101DCC001F4F0E94AA14012B0895E0915E04F0911C
:101DDC005F04089502E0801600E09006A006B006AD
:101DEC000895BEDA59F06EDE4A2F5B2F082F192F9B
:101DFC00E8DF11F401E003C005D0A9F70027E4E007
:101E0C000C94FB164CEC5DE0082F192FC4DD00235D
:101E1C000895A6DA69F056DE4A2F5B2F082F192F8A
:101E2C000E940617012B11F401E003C0EBDF99F7B8
:101E3C000027E4E00C94FB1693DA61F0E82FF92FFD
:101E4C000DD0EA2FFB2F97DC4ADC11F401E003C024
:101E5C00D9DFA1F70027E4E00C94FB16008511856F
:101E6C002285338508959A938A932F9700271127FB
:101E7C00222733273DDC09F472C02EE032E0EEE07D
:101E8C00F2E0E250FE4F0081118105351A4A09F04B
:101E9C0066C022543E4FE22FF32F04810093380486
:101EAC00DDDF26DC09F45BC08EE092E000913804A3
:101EBC00045029F0025019F0065029F150C054D0AA
:101ECC00438554856BD041875287638774874587D8
:101EDC0056876787708BE82FF92F0681178144E0AE
:101EEC000E94E315177F40914A0455270E94EA157A
:101EFC000093490431DCE8E3F4E0418552856385C5
:101F0C00748537DC2AC030D0418D528D47D0458343
:101F1C0056836783708701E000934904E82FF92FFB
:101F2C0001A112A123A134A1023081DA30F001A168
:101F3C0012A123A134A1ACDA01C0B4DADADBF2DAF3
:101F4C00088719872A873B8700270C870D8746D07F
:101F5C00202F212B11F00093490401E001C0002730
:101F6C002F968991999108950B96E82FF92F418915
:101F7C005289638974890381148122273327400F86
:101F8C00511F621F721FE8E3F4E0418352836383A5
:101F9C007483E82FF92F0581112708950E94CC1521
:101FAC00228120934A044189528963897489038070
:101FBC001480400D511D631F731F2227400F511FAA
:101FCC00631F721FE8E3F4E008950C2F1D2F085FC8
:101FDC001F4F1A930A9345E352E008950C2F1D2FBF
:101FEC00085F1F4FBCCA9A938A9300E410E020E06C
:101FFC0030E07EDB51F18EE092E00EE012E00E94C8
:10200C004415013011F505E05EDD4CE452E00EE0C4
:10201C0012E00F5FD5DEC9F40FE7009338040EE031
:10202C0012E004561F4FC0DEE8E3F4E062DB805B95
:10203C009F4F082F192F0E946F1542E00E941C160B
:10204C00EBE4F4E09DDB01E001C00027899199915C
:10205C0008959A938A93992781E0863038F4082F53
:10206C000AD00CD00CF493958395F7CF092F899156
:10207C0099910895082DE5C9402F512FEC5EFB4F27
:10208C000081003008959A938A93239763D000912E
:10209C0038040F3721F55CDC83DE0030184020401B
:1020AC003040A9F555DC25DD91F50C2F1D2F1A9329
:1020BC000A93482F592F4CDC89DC002341F1E09125
:1020CC005B04F0915C04018D01FF21C0E82FF92F16
:1020DC000685046060DE3CDC67DE43D036C075DE0E
:1020EC00028D138D44895589242F352F4081453E0F
:1020FC0071F04081442359F0438544FF08C0448D5E
:10210C00558D668D778D452B462B472B11F000276F
:10211C001DC044275527E82FF92F448745870230E7
:10212C0014072407340728F081D940914A04B4D904
:10213C0001C0B8D9E82FF92FC4DC40915E0450914E
:10214C005F04082F192F0E942A1701E0239689910A
:10215C0099910895802F912F0FE010E01A930A9314
:10216C0003C0E82FF92FC8CC44275527082F192F67
:10217C000C94411706DD49E450E1F2DB002331F009
:10218C00E82FF92F06850260068703C00FE09BDC61
:10219C00EBDF01E0899199910895F3DC49E450E17A
:1021AC00FADB002331F0E82FF92F06850260068751
:1021BC00F0CF0FE088DCD8DFECCFE02FF12F2685B5
:1021CC0021FF06C04BDEE8E3F4E09FDA01E008955E
:1021DC00002708959A938A93BDDFE8E3F4E0058520
:1021EC00168527853089418552856385748577DA14
:1021FC0069DC19F44AE352E002C043E452E0082FD0
:10220C00192F0E94DC14E8E3F4E005851685278578
:10221C003089A7DF068502600687BBCF05E414E092
:10222C000C94AA15AEDCFDD821F211D069F04ADC71
:10223C0048E252E0082F192FC4DD31F0E82FF92FB6
:10224C00068500680687A5CFDDDD79F7B2CF082FAC
:10225C00192F085F1F4F83D9012B089592DCD2DD13
:10226C0009F4A7CFF4DFD9F32DDC48E252E0082FB4
:10227C00192FA7DDA1F3E82FF92F06850068068733
:10228C0088CF97CF0E94EA16802FA42FB52F0FE08E
:10229C001ADC442755270A2F1B2F0E94411788232D
:1022AC00C1F08630B0F400911404083091F4082F7A
:1022BC00E2DEE2DE64F4425F5B4F0A2F1B2FBCDDD3
:1022CC00002329F0EA2FFB2F06850068068701E022
:1022DC0001C00027E4E00C94FB160E94E5162F9732
:1022EC00802E442E552E002309F47BC006E0801668
:1022FC0008F077C000911404083009F072C0485FF0
:10230C005F4F0C2F1D2F98DD002309F46AC0E5E503
:10231C00F4E080819181A281B38160DE012B09F40C
:10232C0060C0009138040F3709F459C0DDD909F4A5
:10233C0058C0E42DF52D068548DD02FF03C003854A
:10234C00016002C003850E7F0387082F192F53D01D
:10235C0009F447C0082D4AD0202F312F025F1B4FA4
:10236C00EC2FFD2F389647E050E00E94BB16E22F71
:10237C00F32FEC5EFB4F008100680083E42DF52DFC
:10238C0006852C5E3B4FE22FF32F02FF03C000812A
:10239C00046002C000810B7F0083A1E0A630F8F43A
:1023AC000A2F24D0802F912F825F9B4FE82FF92F7B
:1023BC0040805180628073805DDEE25FFB4F1AD8F3
:1023CC00401651066206730641F4A81531F0082F29
:1023DC00192F47E050E00E94BB16A395DFCF01E018
:1023EC0001C000272F96E9E00C94F616112747E060
:1023FC0050E00C94CC152A2F3B2F30D80023089595
:10240C009A938A93202F0023A9F0263098F40091F8
:10241C001404083079F407E056DB5527022F47E007
:10242C000E94CC15025F1B4F40E050E00E94411708
:10243C0001E001C00027899199910895002321F0B2
:10244C00063010F401E0089500270895002369F088
:10245C00063058F410DE12DE44F406FF03C000E030
:10246C0011E0089500E810E0089500271127089561
:10247C00002379F0063068F4FEDDEC5EFB4F208122
:10248C0020303CF40E5E1B4FE02FF12F00811181A8
:10249C0008950027112708950E94E6162F970091A2
:1024AC0038040F3709F455C0D4DD11274DE050E046
:1024BC000E94CC15802F912F48E252E00C2F1D2F3B
:1024CC0090DC002309F445C0AA277FDC848F958F0C
:1024DC00A68FA78F0E94FE0990DFD9F148845984FA
:1024EC006A847B8488279927A1E0A63080F50A2F7F
:1024FC00C2DDC2DD54F5425F5B4F0C2F1D2F9CDCFF
:10250C00002319F19DD8F4D821F104E427D00A2F27
:10251C00005D24D00DE322D0D5DA4C2F5D2F4E5F19
:10252C005F4F082F192F025F1D4F0E942A17089624
:10253C000DE014D00AE012D00027E82FF92FE25F4B
:10254C00FD4F00837DD859DF21F0A395CECF01E05C
:10255C0001C000272F96E8E00C94F716E82FF92F0E
:10256C000196E25FFD4F00830895EBE4F4E04AE04E
:10257C0050E00C94BB1605DB00913804E82FF12FCA
:10258C00008300914A04018364DDE82FF92F028354
:10259C0002E303838991999108950E94E016802E9D
:1025AC00A42EB52ECE84DF84002309F464C006E08B
:1025BC00801608F060C05EDDEC5EFB4F80818030E1
:1025CC000CF059C057DDEE5EFB4F008111810A15EE
:1025DC001B0508F450C00A2D0B2909F44CC086FFCA
:1025EC0004C0662401E0702E03C000E8602E77243E
:1025FC0046D00A2D1B2D0E94BD090A2D1B2D01D979
:10260C0071F076D8C1F10A2D1B2DEFD8005F1F4F4A
:10261C007A926A92025F1D4F402F512F26C068D8C4
:10262C0051F100E112E006191709262D372D205122
:10263C0030403A932A93025F1D4F402F512F0C2D9F
:10264C001D2D0E942A178F5F9F4FAF4FBF4F4CD845
:10265C0091F0062D172D0051104020E130E03A93F7
:10266C002A934EE052E0C00ED11E0C2D1D2D0E945F
:10267C002A1701E001C00027E0E10C94F11600E0FC
:10268C0012E0462D572D0E94EA15402E512E08952A
:10269C000E94DE16802EC42ED52EE888F988009173
:1026AC0038040F3709F471C0882009F46EC006E0B5
:1026BC00801608F06AC0DEDCEC5EFB4F8081803057
:1026CC000CF063C082FD61C0D5DCEE5EFB4F008177
:1026DC0011810C151D0508F458C00C2D0D2909F499
:1026EC0054C086FF04C0662401E0702E03C000E8CD
:1026FC00602E7724C4DF0C2D1D2D0E94BD09882E61
:10270C00992EAA2EBB2E0C2D1D2D7BD899F00E9434
:10271C007E0BD9F10C2D1D2D68D8802F912F409652
:10272C007A926A9236D00E942A17082D192D63DEF0
:10273C0061F129C00E947E0B41F180E192E0861983
:10274C009709062D172D005110401A930A9321D08A
:10275C00BED953DED1F00FEF801A900AA00AB00A4E
:10276C00862D972D80519040B4D90E947E0B69F034
:10277C0000E1A9D9E80EF91E4E2D5F2D0EE012E0F6
:10278C00A6D93BDE11F001E001C00027E2E10C9478
:10279C00EF164E2D5F2D825F9D4F082F192F089538
:1027AC000E94E9162A97A02FB12F48E252E019DBBC
:1027BC00002309F47CC0EA2FFB2F04851585012B1F
:1027CC0009F075C00AE27FD97ED00EE014E074D017
:1027DC00EEE0F4E00E94000A0E947E0B09F467C050
:1027EC00F4DB0EE012E00E940215802F912F012BDA
:1027FC0009F45DC0E82FF92F0081043409F044C0BE
:10280C0002810D3309F040C0418000ED400EE1F132
:10281C0006E04016C8F5082F192F0D5F1F4F0E94B8
:10282C005F170930104080F54DD940E250E00C2F75
:10283C001D2F0E5F1F4F0E944117082F192F0D5F80
:10284C001F4F0E945F171A930A930396482F592F14
:10285C000C2F1D2F0E5F1F4F0E942A174C2F5D2F20
:10286C000A2F1B2FD6DA002379F00A2F1B2FB8DB87
:10287C00012B29F0EA2FFB2F068500680687042D13
:10288C00B5DD025F1B4F18D0EEE0F4E00E94000AA9
:10289C000E947E0B61F099DB002711270E94021524
:1028AC00802F912F012B09F0A5CF01E001C000274B
:1028BC002A96E5E00C94FA16EA2FFB2F389647E09F
:1028CC0050E00C94BB16442755270EE014E00C94F2
:1028DC0041172F9703E1F7D84427552708E314E055
:1028EC000E9441170AE2EFD8EEDF0BE414E00E94DD
:1028FC005807002331F10A9519F00A9529F021C0E7
:10290C00B2DA002321F41DC06EDB0023D1F005E404
:10291C0014E00E947615002329F00C2F1D2F40DFA8
:10292C00002369F401E414E00E94AA150E94580ADD
:10293C000E948B0B0C2F1D2F33DF002311F001E0B5
:08294C0001C000272F96089539
:04025200FFFFFFFFAC
:100224004154520053494F32494445200043464704
:100234000020090D0A00433A28524F4F5429002840
:0E0244005355424449522900434430303100A2
:1029540028813981622F732F21503040672BD9F0A1
:10296400E02FF12F6081E42FF52FC895601571F0E9
:10297400E02FF12F0081E42FF52FC895001618F4ED
:1029840001E010E00AC00FEF1FEF07C00F5F1F4FF9
:102994004F5F5F4FDFCF002711272296089505D0A0
:1029A4000F5F1F4F008311830895E82FF92F0081D3
:1029B400118108959A938A938A819B81282F392FB4
:1029C4000197232B59F0E42FF52F4F5F5F4FC895E4
:1029D400E02FF12F01920E2F1F2FF0CF89919991A3
:1029E40022960895E02FF12FC895002031F0C89564
:1029F400041629F00F5F1F4FF5CF00271127089504
:102A04000E94E816442E552E8E819F81202F212B63
:102A140021F0E82FF92F00831183C7DF012B41F048
:102A24002BD021F020D011F0BADFFACF25D019F441
:102A34000027112715C0E82FF92FA081B1811CD0E0
:102A440069F011D011F4ABDFFACF0027E82FF92F8A
:102A540020813181E22FF32F0083A1DF0A2F1B2F66
:102A6400E8E00C94F916A1DFE02FF12F4081042D4A
:102A7400152DB8DF012B089598DFE02FF12F008189
:042A8400002308958E
:102A8800E02FF12F00810895E02FF12F0081112709
:102A98000895E02FF12F008111810895E02FF12F83
:102AA80020810181122F0895F4CFF3CF402F512FA9
:102AB800E02FF12F0081302F22271127E42FF52F47
:102AC8000180322E202D33290280312E102D3329FA
:102AD8004381042F0895E02FF12F00811181228175
:042AE8003381089599
:102AEC00E02FF12FE199FECF19D0E09A0DB30A3AFD
:102AFC0091F4E199FECF05E61BD0E199FECF06E6F5
:102B0C0017D0E199FECF07E613D0E199FECF08E686
:102B1C000FD001E0089500270895F89404E610E022
:102B2C001FBB0EBB089510E01FBB0EBB019107C06D
:102B3C0010E01FBB0EBBE09A0DB3019308950DBBC3
:102B4C00E29AE19A78940895E02FF12FE199FECF63
:102B5C00E4DF0FEFF4DFE199FECFF89405E6E3DF55
:102B6C00E199FECFF89406E6DEDFE199FECFF8940A
:102B7C0007E6D9DFE199FECFF89408E6D4DFE199B6
:0C2B8C00FECFCBDF0AEADBDF01E008959A
:102B9800002411240030010741F01695079510F420
:102BA800040E151E440F551FF5CF002D112D089545
:0E2BB8004A9522F0000F111F0C94DC150895B1
:0E2BC6004A9522F0169507950C94E315089594
:102BD40000241124E0E1EA9552F0001F111F001CAB
:102BE400111C04161506B8F3041A150AF4CF001FB5
:0C2BF400111F402D512D009510950895E3
:102C00000024112422243324E02FE12BE22BE32B98
:102C100071F0369527951795079520F4040E151E2B
:102C2000261E371E440F551F661F771FEDCF002D40
:082C3000112D222D332D089512
:102C38004A9532F0000F111F221F331F0C941C16E7
:022C48000895ED
:102C4A004A9532F036952795179507950C942516CF
:022C5A000895DB
:102C5C000024112422243324E0E2EA9592F0001F90
:102C6C00111F221F331F001C111C221C331C0416A5
:102C7C0015062606370688F3041A150A260A370A9B
:102C8C00ECCF001F111F221F331F402D512D622D21
:0C2C9C00732D009510952095309508953B
:102CA800C895702D3196C895602D3196C895502DD0
:102CB8003196C895402D3196C8953196102C01FA59
:102CC800C8953196202CC8953196302C0895F1DF9F
:102CD800041B10E003C0EADF041B150B20E030E002
:102CE80005C0DEDF041B150B260B370BC8F010FCE4
:102CF8001AC03AD0402D38D00417100588F446F48D
:102D0800E00FF11FC895E22DF32DE019F04009946A
:102D1800000F111FE00FF11F27D0202C25D0302CD9
:102D2800E22DF32D099411F4BEF7ECCF31960EF095
:102D3800319650E060E070E017D0402D4B3F68F0CE
:102D480079F34F3F41F04E3F21F00ED0702D0CD05B
:102D5800602D0AD0502D08D0402D041B150B260BD2
:0E2D6800370B11F3E8F2E2CFC89531960895CB
:102D7600BF93AF93A02FB12F02C001900D92415087
:0A2D86005040D8F7AF91BF910895B7
:102D9000BF93AF93A02FB12F03C0C89531960D926A
:0C2DA00041505040D0F7AF91BF91089512
:0E2DAC00002401C0019201501040E0F708958C
:022DBA00000017
:102DBC00FA92EA92DA92CA92BA92AA929A928A9267
:102DCC007A926A925A924A92BA93AA939A938A9353
:022DDC00089558
:102DDE00FF84EE84DD84CC84BB84AA8499848884A9
:102DEE007F806E805D804C80BB81AA8199818881B5
:0E2DFE00F0E00FB6F894CE0FDF1F0FBE089561
:102E0C0028813981622F632B79F0E02FF12F6081BB
:102E1C00E42FF52F7081671739F40F5F1F4F4F5F49
:102E2C005F4F21503040EECF232B51F0E02FF12F8C
:102E3C0000811127E42FF52F2081021B104002C0C6
:082E4C000027112722960895CA
:102E540068817981202F312F062E172E6150704002
:102E6400012859F0E42FF52F0080E22FF32F01926F
:0E2E74002E2F3F2F4F5F5F4FEFCF2296089516
:102E82009A938A938A819B81E02FF12F282F392FE1
:102E92000197232B11F04193F9CF899199912296B1
:022EA200089591
:102EA400E02FF12F3081341739F021910E2F1F2F8D
:0A2EB4002223B1F70027112708952B
:102EBE00E02FF12F2081222311F03196FBCFE01B62
:082ECE00F10B0E2F1F2F0895D8
:00000001FF
